:030000000210D219
:03000B000200A24E
:03002B00020309C4
:03005B0002047E1E
:0300730002044D37
:1000800002030406080C10182030406080040608A3
:100090000C10182030406080A0C005050D0503033A
:1000A0000302306306C26385768A32C2AFC0D0C015
:1000B000E020623720680241E530660241A5302F1A
:1000C00002E4730563C37405952540F5956340F11B
:1000D0002069EE758A00758D00E525700B758A0024
:1000E000758D00D263757600020302C3E5253340A7
:1000F00009758A00D263F57601FCF58AC262E525AE
:10010000F47002216C2068022153207213758B0059
:10011000758D00D0E0D0D0D293D297D295D2AF32A5
:10012000D293D297D295740CD5E0FDE53C1420E231
:100130001520E10D207D02D296307D02D29202017F
:1001400066D294020166207D02D292307D02D29660
:10015000020166758B00758D00D0E0D0D0D293D2AD
:1001600097D295D2AF32758B00758D00D0E0D0D08C
:10017000D2AF3241E5E525600A207D02C293307D91
:1001800002C297D29541E5E5256002C295207D0225
:10019000D297307D02D29341E5E525600A207D02A9
:1001A000C297307D02C293207D02D293307D02D26D
:1001B0009741E5207D02C292307D02C296207D02E9
:1001C000C296307D02C2927414D5E0FDE525600A26
:1001D000207D02C293307D02C297D29541E5207DF9
:1001E00002C292307D02C296C2947414D5E0FDE53D
:1001F00025600A207D02C293307D02C297D29541CC
:10020000E5C294207D02C292307D02C2967414D55C
:10021000E0FDE5256002C295207D02D297307D0287
:10022000D29341E5C294207D02C296307D02C292F3
:100230007414D5E0FDE5256002C295207D02D297B9
:10024000307D02D29341E5207D02C296307D02C20C
:1002500092C2947414D5E0FDE525600A207D02C2A7
:1002600097307D02C293207D02D293307D02D297D7
:1002700041E5207D02C296307D02C292207D02C2FD
:1002800092307D02C2967414D5E0FDE525600A2007
:100290007D02C297307D02C293207D02D293307DD1
:1002A00002D29741E530723DE53C20E21A20E12977
:1002B000207D02C292307D02C296207D02C296301D
:1002C0007D02C2920202E520E1E6207D02C2923068
:1002D0007D02C296C2940202E5C294207D02C296BB
:1002E000307D02C292E525F4C3334009758A00D2FD
:1002F00063F57641F7F58A758B00758D007563009F
:10030000D262D0E0D0D0D2AF32C2AFC2AD53E6EFAE
:10031000C0D0C0E0D2D3D2AFE5776009E574600504
:1003200075740061F8757401C2CEE5296007207408
:10033000461529617778007900E580307E01F43038
:10034000E50278FF53DACF207E0343DA20307E03C4
:1003500043DA10C2D8C271E580307E01F430E50284
:1003600079FFC3E89970CE306103752918207403B2
:100370007529188859D270E52A6004152A618720EA
:10038000740543DA01C2D820700261E2A8592061E5
:1003900002C270207431C3E894F0400374F0F8E8AE
:1003A000C4540F28F87984B7030261C7C313C31379
:1003B0008721200802C313200A06C3C898F861C722
:1003C00028F8500374FFF8C3E895625003E562F81B
:1003D000882230690AC3E522955E4003855E228546
:1003E0002224A824C3E524955E4002A85E8825C384
:1003F000E52594404002D26420CF0CD0E0D0D0C29A
:10040000D343E610D2AD32E5776009E57560057536
:1004100075008141757501C2CF7801E5296005300D
:1004200074021529C3E55994014005755C008141AA
:10043000755D00756400E55C2401F55C5003755C36
:10044000FFD0E0D0D0C2D343E610D2AD32C0D0C08E
:10045000E0C2AF53917F53E67FC260C3E55033F5EE
:1004600050E55133F551759100C3E49550F594E48E
:0E0470009551F595759104D0E0D0D0D2AF3201
:10047E00C2AF53E6EFC2ADC0D0C0E0C0F0D2D3D20F
:10048E00AFA8FBA9FCE5776007C3E913F9E813F8F9
:10049E00C2D830710281F053DACF207E0343DA10D6
:1004AE00307E0343DA20D271E580307E01F420E500
:1004BE000281C788268927E12C53DACF207E034399
:1004CE00DA20307E0343DA10C2D8C271307402E1F2
:1004DE00187800E580307E01F430E502E118885985
:1004EE00C1FF53DACF207E0343DA20307E0343DA96
:1004FE0010C271206102A1C053DACF207E0343DA0D
:10050E0010307E0343DA20C2D8D27188548955C385
:10051E00E89552F8E99553F9E4FB7E027A00C3E8B8
:10052E00948CE994005005755800A1B0C3E894C8A6
:10053E00E994005008E4D2E4FB7A0AA18DC3E89452
:10054E0068E994015008E4D2E3FB7A0FA18DC3E869
:10055E0094D0E994025008E4D2E2FB7A1EA18DC336
:10056E00E894A0E994055008E4D2E1FB7A3CA18D11
:10057E00C3E89498E994085008E4D2E0FB7A787EB8
:10058E0000C3E89556FCE99557FD30E708ECF424D6
:10059E0001FCEDF4FD755800C3EC9AED9E50037509
:1005AE00580188568957A854A955885289537802FC
:1005BE00C1FFC3E89526F8E99527F9307C02C1E31F
:1005CE00307B02C1E3307A02C1DC207502A1E3E97F
:1005DE00FDE8FCC102E9C313F9E813F8307902C152
:1005EE00DCE9C313F9E813F8307802C1DCE9C31370
:1005FE00FDE813FC206126C3EC941CED940240022E
:10060E00C119ED7018C3EC94C850120528C3E52823
:10061E00940A5002E118755900D270E118E528606D
:10062E000215287400207F0B7888E67896B40302B2
:10063E00789EE624FAFEE43400FFC3EC9EFCED9FA8
:10064E00FD92087888E6B40327A2085009207D2081
:10065E00C2AFD27DC16B307D17C2AFC27DD293D2F5
:10066E0097D295C292C296C294206902D26BD2AF33
:10067E00A2085017E6B4030DECF42401FCEDF4349B
:10068E0000FD02069978007900C1E37888E6B4038C
:10069E0015EC33FCED33FDC3EC940AFCED9400FD38
:1006AE0050047C007D00C3EC94FFED94004006786E
:1006BE00FF7900C1E3EC856FF0A4C5F0A2F733F823
:1006CE00790040030206FF78FF79000206FFE9C3B6
:1006DE0013F9E813F8307C0EE9600278FFC3E813D3
:1006EE0038F8E43400F9C3E894FFE9940040027846
:1006FE00FF8859D270206102E118741FF4552F4BF8
:10070E00F52FC274E42B7002D2747529183074035D
:10071E0075290A306102E12C20740353DAFE752A22
:10072E0006307403752A0AD0F0D0E0D0D0C2D3D2EE
:10073E00AD43E61032790102076179030207617950
:10074E000A020761791E020761796402076179C89E
:10075E000207617817E4D5E0FDD8FAD9F6227A14AB
:10076E007B780207887A107B8C0207887A0D7BB41F
:10077E000207887A0B7BC8020788AC25752501799C
:10078E0002B27DE4C294D5E0FDE5256002C295D5A6
:10079E00E0FDD295D5E0FDD294D5E0FDE525600AC9
:1007AE00207D02C293307D02C297E570D5E0FD2018
:1007BE007D02D293307D02D2977496D5E0FDD9C1D9
:1007CE00EAF8D5E0FDD8FBDBB1C2948C2522C37CC0
:1007DE00007D0075F00005F0EA33FAEB33FB50F6BE
:1007EE00EB13FBEA13FAC3E9FFE8FEE89AF8E99B7C
:1007FE00F95004EFF9EEF8B3EC33FCED33FDD5F020
:10080E00DFEDF9ECF822E889F08A20D2D4F8A9F0CD
:10081E007B0030F70B7BFFF42401F8E9F43400F988
:10082E00E88520F0A4ADF0F8E98520F0A4AFF0FE45
:10083E00ED2EF974003FFA7C04C3EA13FAE913F9BA
:10084E00E813F8DCF48BF030F70AE8F42401F8E949
:10085E00F43400F9E889F0C2D4F8A9F02222E54771
:0F086E00603BC3E53B13F9E53A13F8C3E53E9849
:10087D00F8E53F99F9500CC3E89480E994FF4016D0
:10088D000208A7C3E8947FE9940050030208A778F3
:10089D007F79000208A7788079FF8843894422E593
:1008AD00476058E5432540F8E5443541F985442036
:1008BD00E4300701F43542FA30E709C3EA94F04019
:1008CD00150208E9C3EA940F50030208E978FF798D
:1008DD00FF7A0F0208E9780079007AF0C3E52495D4
:1008ED005E5006E52460092102E54420E70D210252
:1008FD00E54430E706884089418A4222E547700386
:10090D0002096C78A1E6FAC3E54333F8E54433F9FF
:10091D001114E930E70BC3E89480E994FF401321EB
:10092D0043C3E8947FE9940050022143787F790016
:10093D002143788079FFE820E715C3E52398F84037
:10094D0009C3E89401400302096A780102096AE8C3
:10095D00F424012523F8400302096A78FF88452213
:10096D00E54770030209CE78A2E6FAA841A9421123
:10097D0014E930E70CC3E89401E994FF401602092D
:10098D00A5C3E894FFE9940050030209A578FF7907
:10099D00000209A5780179FFE920E715C3E545981F
:1009AD00F84009C3E8940140030209CC780002091C
:1009BD00CCE8F424012545F840030209CC78FF88E2
:1009CD00242278FFC264E52D5406702FD264C3E54E
:1009DD003B940A4009C3E52594405002C264E53BAF
:1009ED00601974FF853BF0848537F0A4F8C5F0607D
:1009FD000278FFC3E895615002A861886022020A5F
:100A0D00A87883E6F520120EF375E890120743756A
:100A1D00E890E5E820ECFBA8BDA9BE120F89756B27
:100A2D0001756C00C3740013FD740113FC74012C6B
:100A3D00FC74003DFDECFAEDFBC3E89AE99B401414
:100A4D00E56B2401F56BE56C3400F56CEA2CFAEBE3
:100A5D003DFB80E5AE6BAF6CC3E56C13F9E56B1335
:100A6D00F8C3E913F9E813F8E56B28F569E56C3976
:100A7D00F56A7A03C3E913F9E813F8DAF7AA201A2D
:100A8D007009756B00756C00020AA81AEA6008EE11
:100A9D0028FEEF39FFDAF88E6B8F6C2275E8902205
:100AAD007883E6FFE5E820ECF7A8BDA9BE056DC388
:100ABD00E56D94084052756D00E9FA79A0E7604440
:100ACD00EA7007E56E601B020AE3C3E8956E6010DD
:100ADD00E56E5006600C14020AEF0460F9020AEF8D
:100AED00E56EF56EC39472401B755EC0C3940440F1
:100AFD0013755E80C39404400B755E40C39404402F
:100B0D0003755E0075BB0822E55EF46002055EE5C7
:100B1D006DB4070375BB1022743279A387F0A4C599
:100B2D00F0A2F733F8C3E8955E4002A85E882288EC
:100B3D00248825886122753A00753B7F2275C8206F
:100B4D00A8CCA9CD75C824C3E913F9E813F8AA38C0
:100B5D00AB3988388939C3E89AF8E99B547FF9AAEB
:100B6D003AAB3BAC3AAD3B7E047F02C3EB94044001
:100B7D00021E1FC3EB940840021E1FC3ED13FDECB4
:100B8D0013FCDEF7C3EA9CFAEB9DFBEF6009C3E9AA
:100B9D0013F9E813F8DFF7EA28FAEB39FB8A3A8BF9
:100BAD003B400122753AFF753BFF2230600261B870
:100BBD00854C50854D51D26043E680227892E6FFF8
:100BCD00C3E535948240010FC3E53594A040010F74
:100BDD00C3EF940640027F057E021E3072010EC3E4
:100BED00E53B940350060E0E3072010EC3E53B94A7
:100BFD000250060E0E3072010EA93BA83A7A04C3BC
:100C0D00E913F9E813F8DAF7C3E89EF8E99400F967
:100C1D004009C3E89402E9940050047802E4F9E92C
:100C2D00FBE8FAC3E913FDE813FC884C894DC3EFCB
:100C3D0094036037EF20E00DE82CF8E93DF9ECFA6C
:100C4D00EDFB020C65E828F8E939F9C3E89402F8E0
:100C5D00E99400F97A02E4FBC3EF9403400D8A4E48
:0F0C6D008B4F884889498C4A8D4B22884E894F7E
:100C7C008A488B498C4A8D4B223060028185D26028
:100C8C0043E680E52D5406602EA83AA93BE5349442
:100C9C00085006E820E002A94DC3E833F8E933F91F
:100CAC00759100C3E498F594E499F595759104D287
:100CBC006053917F43E68022D265753D007520001C
:100CCC00020CD7D265753D00752040E52D540660A9
:100CDC0002C265D2AF206005E53D60012278017A41
:100CEC0002C3E53B940540027802C3E53B940A40FD
:100CFC00027803C3E53B940F40027A033069047811
:100D0C001E7A01206007E53D6003D2AF22D2AF000E
:100D1C0000C2AFC3E53BFB940F40027B0FEB0430EA
:100D2C0073012320620123F93069027982E58D1366
:100D3C00E58B13C39940CC053DEAFBE59B5440B5CC
:100D4C002004DBF7A17D20650281D7C26575910077
:100D5C00AE3AAF3BC3EE33FEEF33FFC3E49EF594E4
:100D6C00E49FF595759104D26053917F43E68081A1
:100D7C00D730650281D7D88BD2AF2230690B0534BE
:100D8C00206016753400020DA520600D20650A2028
:100D9C006B07158115810215A922A84EA94FC3E82E
:100DAC0033F8E933F975910053917FC3E498F594C6
:100DBC00E499F595759104854850854951D2604365
:100DCC00E6802278003064053065027801E53575DF
:100DDC00F007A4F9E5F028F5F0E9A2F013A2F1135D
:100DEC00A2F213F535C394785003753578C3E53505
:100DFC0095364008D266D293D297D295306002C114
:100E0C0008854A50854B51D26043E68022C2AFC25E
:100E1C0092C296C29430720B9002477414D5E0FDC6
:100E2C00020E2F207D02D292307D02D296759F4009
:100E3C00753C02020F6EC2AF207D02D297307D024C
:100E4C00D293307217900224C294207D02C2963045
:100E5C007D02C2927414D5E0FD020E6B90018730B6
:100E6C006206E5256002C295207D03759F41307DA9
:100E7C0003759F43753C03020F6EC2AFC292C296BC
:100E8C00C29430720B9002017414D5E0FD020E9CDA
:100E9C00207D02D296307D02D292207D03759F4335
:100EAC00307D03759F41753C04020F6EC2AFD29525
:100EBC003072179001DE207D02C292307D02C29604
:100ECC00C2947414D5E0FD020ED990017530620EF7
:100EDC00E525600A207D02C293307D02C297759F82
:100EEC0040753C05020F6EC2AFC292C296C29430DE
:100EFC00720B9001B37414D5E0FD020F09D294204B
:100F0C007D03759F41307D03759F43753C06020F31
:100F1C006EC2AF207D02D293307D02D29730721F09
:100F2C00900272207D02C292307D02C296207D0218
:100F3C00C296307D02C2927414D5E0FD020F4E9021
:100F4C00019930620EE525600A207D02C297307D42
:100F5C0002C293207D03759F43307D03759F4175BD
:100F6C003C01306B13120F897414D5E0FD740CD551
:100F7C00E0FDD292D296D294C266D2AF2290017387
:100F8C00D293D297D295C292C296C294C262227860
:100F9C008076FF0876FF0876FF0876FF0876030850
:100FAC00760408760B087603087601087601788CAF
:100FBC0076010876FF0876FF0876FF0876FF08763C
:100FCC00FF0876030876FF0876FF0876FF0876257B
:100FDC000876D00876FA0876FA0876040876FF08C0
:100FEC00760108760008767A0876FF087601227872
:100FFC0087E6FFC272BF0302D2727888E6C39403FD
:10100C006008C27DE630E102D27DC27E7889E6308E
:10101C00E102D27EC3EF94026008758E01D2730296
:10102C001033758E00C273227880E6149000809382
:10103C0078A1F67881E6149000809378A2F6120FCE
:10104C0089227886E61490008D9378A3F6120F8986
:10105C002222789CE67536FF75370CB4020675367D
:0F106C00A075370AB40306753682753705222240
:10107B007896E6FA7897E6FB307F047A007BFFC31D
:10108B00EB9AFCC3948250027C82756F00056FEC67
:10109B00856FF0A4C3E5F0948040F222D27F117BE0
:1010AB001207527A007B007C10120748E5592AFA86
:1010BB0074003BFBDCF37C04C3EB13FBEA13FADC9D
:1010CB00F7FEC27F117B22E5EF20E60375200005BA
:1010DB0020903FFFE520146006901FFF14600093E3
:1010EB0004600375EF12C2D353D9BF7581C043FFA0
:1010FB008012074375EF0243B203E5B3240420E7E4
:10110B0002F5B3120F897580FF75A40075F1307568
:10111B00D4DF7590AB75A5FC75F2FC75D50175A682
:10112B000175E241120F9B1215E478988670C2AFDD
:10113B0012075C12076C1207521207731207521236
:10114B00077A1207521216F812075C12075C120785
:10115B0057C2AFE4F8F6D8FD78C879C8308507D9FF
:10116B00FBD8F7021C00120F9B1215E4120FFB1198
:10117B0034114E115D115E117A117B7898867012C5
:10118B000F8975B68075A9007577007588507589BC
:10119B001275C82475910475D84075A82275B802CC
:1011AB0075E690759B80759D0075D10E75BCC075ED
:1011BB00BB0875BA1175E880120743D2AF120A0B40
:1011CB0043DA01C2D8C27112075C753001D2617B60
:1011DB00037A0CE55870067A0CDB02215C1207527D
:1011EB00207002215CC270E559C3940240E3E52FE5
:1011FB00541F855B5AF55BB55AD7DAD7C26153DA00
:10120B00CF207E0343DA20307E0343DA10C2D8C2EC
:10121B0071C275752800120757307409C3E52894FD
:10122B000A4002D27512074878023074027800C364
:10123B00E5599840F0C2AF12076C12076C12076C9D
:10124B00D2AF12075C7546007888E6B40302612FB3
:10125B00120748788CE6C39401500302132FE53034
:10126B00C39401500302132F207435C3E55994FF27
:10127B00500302132FC2AF120781D2AF120757C30D
:10128B00E559940150EFC2AF12076C12074D1207CC
:10129B006CD2AF120757C3E55994FF40E902177D93
:1012AB007F05D27F117B120757C2AFC27F117BAE76
:1012BB0059C3E559947FD2AF4074120743C2AF12A2
:1012CB000781D2AFDFDC11A7C3EE94057897F61236
:1012DB00075C1216261217007F0AD27F117B1207AA
:1012EB0057C2AFC27F117BAE59C3E559947FD2AFC2
:1012FB0050E6120743C2AF12076C12074D12076C70
:10130B00D2AFDFD611A7EE24057896F612075C1242
:10131B00162612172F120757117BC3E55994FF405E
:10132B00F402177DC3E559954640038559461207CC
:10133B005778017988E7B403027805C3E5599840DB
:10134B00024153C2AF120781120781120781D2AF3C
:10135B0012075C753000E4F531F5320531E531F4F7
:10136B0070390532789AE678191460127832146065
:10137B000D787D14600878FA146003753200C3E5AC
:10138B003298401715327531B478998670C2AF1206
:10139B000781D2AF7898867012075712074DE5294F
:1013AB007005307402215C78012074027806C3E565
:1013BB00599840A77888E6C394036003120757E552
:1013CB00297002215CC2AF120F89E4F522F523F5D7
:1013DB0024F525D2AF78858662F53EF53FF540F5CD
:1013EB0041F542F56DF547F52CF52DF535120B430F
:1013FB00756D0875BB10120743120AA9E5E820ECBE
:10140B00FBA8BDA9BEE97001F8886E120AAD756D17
:10141B000875BB107887E6FE7602120FFB7887EE15
:10142B00F6C2AF755EFF120B2585225E85225F85A6
:10143B002260D2AF752201752401752501855D648B
:10144B0075650175B69075A903757701D268D26978
:10145B00753400120EF3120F1D120B43120B4A12AE
:0E146B000BC902147C120F89120FFB756D0065
:1014790075BB08120CCF120D87120DA612086B123C
:101489000DCF120E19120B4A120BB8120BC9120CFE
:1014990085120CC4120D87120DA612086C1209CF01
:1014A900120DCF120E42120B4A120BB8120BC912AF
:1014B9000C85120CCF120D87120DA61208AC120D55
:1014C900CF120E86120B4A120BB8120BC9120C85D9
:1014D900120CC4120D87120DA6120909120DCF1292
:1014E9000EB8120B4A120BB8120BC9120C85120C4A
:1014F900CF120D87120DA612096D120DCF120EF320
:10150900120B4A120BB8120BC9120C85120CC41219
:101519000AA9120D87120DA6120AAD120DCF120FCC
:101529001D120B4A120BB8120BC9120C8530693502
:10153900206B3285615E85615F855D6475650179C2
:10154900327A0AC3E53499400FC269D26A8A33757F
:101559005EFF755FFF02156EC3E5599401400302F2
:10156900147C0215A9306A1B206B18E5331470042A
:10157900C26A8170F533C3E5599401400302147CB2
:101589000215A9C3E55C94825016307404E52960FC
:101599000FC3E53B78F0306B027860985002817C8C
:1015A900C2AF120F897887E6FE7602120FFB7887A1
:1015B900EEF6E4F522F523F524F525F562C2687502
:1015C900B68075A900757700D2AF120743120F894B
:1015D900307406E5297002215C6161901A0D78204A
:1015E900121668E520B45A0CA3121668E520B4A5B2
:1015F90003021606120F9B121626021625901A03CD
:1016090078807B0A121668A308DBF9901A0F788C88
:101619007B15121668A308DBF9901A2422C2AF12AF
:1016290016A7121681901A00740D12166DA3740272
:1016390012166DA3741312166D901A0378807B0A23
:1016490012166CA308DBF9901A0F788C7B15121609
:101659006CA308DBF91216BA121698901A2422E420
:1016690093F622E6438F01538FFD75EF0275B7A5F7
:1016790075B7F1F0538FFE22438F02438F0175EF47
:101689000275B7A575B7F1901A0DF0538FFC22902A
:101699001A0D745AD16D901A0E74A5D16D227A3033
:1016A90079D07820901A40D168E520F709A3DAF7B4
:1016B900227A3079D0901A40E7D16D09A3DAF9225C
:1016C900AB71A872BB01027984BB02027985BB03A5
:1016D900027986BB04027992BB05027987BB0602AF
:1016E900799CBB07027988BB08027989E8F7227CD3
:1016F9000512075CDCFB22C2AF12076C12077312DA
:10170900077A12078112074D12076C120773120725
:101719007A12078112074D12076C12077312077AA2
:10172900120781D2AF22C2AF12078112077A1207BC
:101739007312076C12074D12078112077A12077389
:1017490012076C12074D12078112077A12077312DA
:10175900076CD2AF22AE71AF72C2AF12076C12071B
:101769006C12076C12074DDEF212078112074DDF6A
:10177900F8D2AF22F100D1F8D1F875710175720173
:10178900757300F15E7C05AD5912075CC3ED95597F
:1017990070F5C3E5599401400AC3E55994FF4032F5
:1017A9000217B9D1C9D126F100C2AF75EF12D1F82C
:1017B900DCD50573C3E5739403500280C6D1F805DF
:1017C90072E5711490009A93F808C3E57298500273
:1017D90080AED1F8D1F80571C3E571940950028042
:0D17E9009C120F9BD126C2AF75EF12D1F8F4
:101A00000D0213FFFFFFFF03040B0301015AA501A1
:101A1000FFFFFFFFFF03FFFFFF25D0FAFA04FF01DE
:051A2000007AFF01FF48
:101A40002358526F746F72313041232020202020A0
:101A500023424C48454C492346333930232020202B
:101A60002020202020202020202020202020202076
:101C0000C2AFC2D353D9BF7581C043B20343FF8073
:101C1000752438752503B1BF75EF0275E24043F1B5
:101C20002053A4DFD285780379E67C1075220075F5
:101C30002300901DCC7B0675249875250130850204
:101C4000813D208508D8FBD9F9DCF781AD308508C6
:101C5000D8FBD9F9DCF781ADB17FE493A3C39A60D7
:101C6000028126DBDDB171600281267B08E493FAF4
:101C7000A3B152DBF87A30B152752200752300B15E
:101C800071EAFCEBFDC3ED94FE400EB1718A278B27
:101C900028ED30E0048A828B83B1717AC270D8C398
:101CA000ED94FE601050CEBD0022EC600675200061
:101CB0000200008100A827A9280809D804D90281B8
:101CC000C9B175EA89AAF281BB0D8199C3ED94036C
:101CD0005049EDA2E092007AC5C3E5829400E58305
:101CE000941C5093200010438F02438F0175B7A5B9
:101CF00075B7F1F030001FA827A9280809438F0104
:101D0000538FFDD804D902A11689AAE275B7A5752B
:101D1000B7F1F0A3A103538FFC81757AC1BD030C09
:101D2000E493A3FAB136DCF8B12E81758177AA224B
:101D3000AB23B152EBFAEA6222752608C3E52313FE
:101D4000F523E52213F52250066323A0632201D573
:101D500026EAB1BFB1BF75260AEAF4200102D28596
:101D6000300102C285B1BFC3134002C201D526EBC8
:101D700022B175EAFB208502A175308502A17A7532
:101D80002608AE24AF25C3EF13FFEE13FEB1C3B197
:101D9000BFC3EA133085024480FA30E703632201AF
:101DA000C3E52313F523E52213F52250066323A090
:101DB000632201D526D9E52265236523F52222AECB
:101DC00024AF250E0FDEFEDFFCD20122424C486517
:0A1DD0006C6934373132F3900601DC
:00000001FF
